:100000000C942A000C9445000C9445000C94450077
:100010000C9445000C94BE010C94EB010C941D0251
:100020000C9445000C945C010C9445000C94450024
:100030000C9445000C9445000C943F030C9445002F
:100040000C9445000C9445000C9445000C9445001C
:100050000C94450011241FBECFE5D4E0DEBFCDBF18
:1000600010E0A0E6B0E0ECE1FFE002C005900D92E8
:10007000A43AB107D9F711E0A4EAB0E001C01D929B
:10008000A130B107E1F70C94AD000C940000CF93C0
:10009000DF93CDB7DEB7E7E3F0E08FE18083E4E301
:1000A000F0E08EEF8083E1E3F0E084E08083E2E340
:1000B000F0E088E38083DF91CF910895CF93DF93C1
:1000C000CDB7DEB723970FB6F894DEBF0FBECDBF16
:1000D000F89480E29EE49093FE008093FD001B82E2
:1000E0002FC08B81482F55278B819927880F991F07
:1000F000FC01EB53FF4F808191819C0128513C4FC3
:10010000CA01880F991FFC01E351FF4F31832083FF
:100110002091FD003091FE008B819927880F991F57
:10012000FC01E351FF4F80819181A901481B590BCC
:10013000CA019093FE008093FD008B818F5F8B83BB
:100140008B81883070F2789423960FB6F894DEBFD6
:100150000FBECDBFDF91CF910895CF93DF93CDB781
:10016000DEB727970FB6F894DEBF0FBECDBF0E9453
:1001700047000E943A010E9431030E9480031092BE
:10018000EC008CED92E09093C0008093BF008AE277
:1001900093E09093C2008093C10078948091A8006E
:1001A0008823E1F31092A8000E9429060E946804A7
:1001B0000E94D00600C08091B200813041F480914D
:1001C000EC00882311F40E945E001092B20080912E
:1001D000AB00813021F41092AB000E94FE068091AA
:1001E000A900813011F41092A9008091A8008130FB
:1001F00029F51092A8000E9470061A821CC080E6A1
:1002000090E00E94BA038A8199270E94040487E63D
:1002100090E00E94BA038A819927880F991FFC01F8
:10022000E351FF4F808191810E9404040E94F503F5
:100230008A818F5F8A838A81893008F38091A70041
:10024000813009F0B8CF1092A700B5CFCF93DF93DC
:10025000CDB7DEB7F894E9E5F0E089E180837894E2
:10026000DF91CF910895CF93DF93CDB7DEB7DF91C4
:10027000CF910895CF93DF93CDB7DEB7E3E5F0E0FC
:1002800082E08083EFE4F0E01082EEE4F0E082E0D0
:100290008083EAE4F0E084EF91E091838083E8E4F6
:1002A000F0E080ED97E091838083E9E5F0E089E17B
:1002B0008083DF91CF9108951F920F920FB60F9216
:1002C00011248F93CF93DF93CDB7DEB78091B60023
:1002D0008F5F8093B6008091B600833029F481E06F
:1002E0008093AB001092B6008091EB008F5F8093FB
:1002F000EB008091EB008732C9F581E08093A90083
:100300001092EB008091B5008F5F8093B5008091D3
:10031000B500853029F41092B50081E08093AA00E1
:100320008091B3008F5F8093B3008091B3008436D7
:1003300041F41092B30081E08093A60081E08093A5
:10034000A8008091B300823319F481E08093A80063
:100350008091B4008F5F8093B4008091B4008A30A4
:1003600029F41092B40081E08093A700DF91CF912F
:100370008F910F900FBE0F901F9018951F920F92A4
:100380000FB60F9211242F933F934F935F936F9368
:100390007F938F939F93AF93BF93EF93FF93CF93ED
:1003A000DF93CDB7DEB7E091BF00F091C0000995B3
:1003B000DF91CF91FF91EF91BF91AF919F918F917D
:1003C0007F916F915F914F913F912F910F900FBE51
:1003D0000F901F9018951F920F920FB60F92112435
:1003E0008F93AF93BF93EF93FF93CF93DF93CDB7EB
:1003F000DEB7A2E3B0E0E2E3F0E080818B7F8C9394
:10040000A5E3B0E0E5E3F0E080818D7F8C9381E0AF
:100410008093B1008091A400883019F481E080932A
:10042000B200DF91CF91FF91EF91BF91AF918F918A
:100430000F900FBE0F901F9018951F920F920FB63E
:100440000F9211242F933F938F939F93AF93BF935A
:10045000EF93FF93CF93DF93CDB7DEB72297DEBF45
:10046000CDBFA2E3B0E0E2E3F0E0808184608C9352
:10047000ECE4F0E011821082A8E4B0E08091A400E6
:100480009927880F991FFC01E351FF4F80819181CB
:1004900011969C938E938091A400882339F4A5E350
:1004A000B0E0E5E3F0E0808182608C938091A4006D
:1004B000282F33273A83298389819A8182309105B5
:1004C000C1F129813A812330310554F489819A811F
:1004D000009789F029813A8121303105D9F04EC049
:1004E00089819A818330910599F129813A8124305B
:1004F0003105E9F143C0A8E3B0E0E8E3F0E0808132
:1005000080618C93A8E3B0E0E8E3F0E08081816053
:100510008C9334C0A8E3B0E0E8E3F0E080818E7F04
:100520008C93A8E3B0E0E8E3F0E0808182608C93F4
:1005300025C0A8E3B0E0E8E3F0E080818D7F8C93F4
:10054000A8E3B0E0E8E3F0E0808184608C9316C01B
:10055000A8E3B0E0E8E3F0E080818B7F8C93A8E330
:10056000B0E0E8E3F0E0808188608C9307C0A8E306
:10057000B0E0E8E3F0E08081877F8C938091A40075
:100580008F5F8093A4008091A400893010F01092B6
:10059000A4002296F894DEBFCDBFDF91CF91FF91EA
:1005A000EF91BF91AF919F918F913F912F910F90BC
:1005B0000FBE0F901F901895CF93DF93CDB7DEB786
:1005C0008091B7009091B8000097B1F4E6E4F0E0B4
:1005D000808191819093BE008093BD00AEE4B0E035
:1005E000EEE4F0E080818F7B8C9381E090E090934B
:1005F000B8008093B7002BC0E6E4F0E080819181E1
:100600009093BC008093BB00AEE4B0E0EEE4F0E079
:10061000808180648C932091BB003091BC008091DC
:10062000BD009091BE00A901481B590BCA019093CF
:10063000BA008093B9001092B8001092B700809170
:10064000B9009091BA00909300018093FF00DF9170
:10065000CF910895CF93DF93CDB7DEB7DF91CF91E0
:100660000895CF93DF93CDB7DEB7E7E2F0E01082D5
:10067000E6E2F0E08FEE8083DF91CF9108951F9244
:100680000F920FB60F9211242F933F938F939F9346
:10069000EF93FF93CF93DF93CDB7DEB7E6E2F0E0C1
:1006A00010828091A5009927E4E2F0E02081318159
:1006B000880F991FFC01EB53FF4F318320838091FA
:1006C000A5008F5F8093A5008091A500883010F071
:1006D0001092A500E7E2F0E08091A5008083E6E2B9
:1006E000F0E08FEE8083DF91CF91FF91EF919F91AA
:1006F0008F913F912F910F900FBE0F901F901895E3
:10070000CF93DF93CDB7DEB7E9E2F0E080E18083FD
:10071000E0E4F0E01082EAE2F0E088E18083E0E4E7
:10072000F0E086E88083EBE2F0E082EC8083DF910A
:10073000CF910895CF93DF93CDB7DEB721970FB652
:10074000F894DEBF0FBECDBF8983EBE2F0E080817D
:100750009927807290700097C1F3ECE2F0E08981F4
:10076000808321960FB6F894DEBF0FBECDBFDF9118
:10077000CF910895CF93DF93CDB7DEB726970FB60D
:10078000F894DEBF0FBECDBF9E838D838D819E8189
:10079000DC01FD0101900020E9F73197CF018A1BB0
:1007A0009B0B9C838B831A8219820FC029813A810B
:1007B0008D819E81F901E80FF91F80810E949A03C3
:1007C00089819A8101969A83898329813A818B81D3
:1007D0009C818217930750F726960FB6F894DEBFD8
:1007E0000FBECDBFDF91CF910895CF93DF93CDB7EB
:1007F000DEB780916A000E949A0380916B000E948C
:100800009A03DF91CF910895CF93DF93CDB7DEB7F1
:1008100066970FB6F894DEBF0FBECDBF9E8B8D8B53
:100820008D899E894AE050E09E012F5F3F4FB901BC
:100830000E944907CE0101960E94BA0366960FB640
:10084000F894DEBF0FBECDBFDF91CF910895CF9357
:10085000DF93CDB7DEB722970FB6F894DEBF0FBE99
:10086000CDBF8A8387E089831FC08A81482F55279F
:100870008981282F332727FD309581E090E0022ED3
:1008800002C0880F991F0A94E2F784239523181653
:10089000190624F481E30E949A0303C080E30E94B6
:1008A0009A0389818150898389818823F4F6809114
:1008B0006A000E949A0380916B000E949A0322961C
:1008C0000FB6F894DEBF0FBECDBFDF91CF91089574
:1008D000CF93DF93CDB7DEB70E94A10463E080E041
:1008E0000E9405068CE690E00E94A70562E081E088
:1008F0000E94050687E790E00E94A7050E949704E2
:10090000E0E3F0E080819927807290700097C1F752
:100910000E94A104DF91CF910895CF93DF93CDB7CB
:10092000DEB78DE00E94DC05DF91CF910895CF9373
:10093000DF93CDB7DEB78CE00E94DC05DF91CF916D
:100940000895CF93DF93CDB7DEB781E00E94DC0539
:10095000DF91CF910895CF93DF93CDB7DEB7269780
:100960000FB6F894DEBF0FBECDBF9E838D838AE0A5
:1009700090E09C838B831CC082E390E09A83898300
:100980000EC08D819E8101979E838D838D819E8176
:100990000097B9F789819A8101979A838983898120
:1009A0009A81009799F78B819C8101979C838B8317
:1009B0008B819C81009701F726960FB6F894DEBFD5
:1009C0000FBECDBFDF91CF910895CF93DF93CDB709
:1009D000DEB721970FB6F894DEBF0FBECDBF898377
:1009E0008981992781709070882341F0A5E3B0E058
:1009F000E5E3F0E0808180618C9307C0A5E3B0E07F
:100A0000E5E3F0E080818F7E8C9389819927827065
:100A10009070009741F0A5E3B0E0E5E3F0E080815D
:100A200080628C9307C0A5E3B0E0E5E3F0E080814D
:100A30008F7D8C938981992784709070009741F005
:100A4000A5E3B0E0E5E3F0E0808180648C9307C02B
:100A5000A5E3B0E0E5E3F0E080818F7B8C938981B2
:100A6000992788709070009741F0A5E3B0E0E5E326
:100A7000F0E0808180688C9308C0A5E3B0E0E5E3F6
:100A8000F0E090818FE789238C9321960FB6F8943C
:100A9000DEBF0FBECDBFDF91CF910895CF93DF931F
:100AA000CDB7DEB7A5E3B0E0E5E3F0E08081846098
:100AB0008C9381E090E00E94AB04A5E3B0E0E5E315
:100AC000F0E080818B7F8C93DF91CF910895CF935D
:100AD000DF93CDB7DEB722970FB6F894DEBF0FBE17
:100AE000CDBF8A838A8182958F70898389810E9494
:100AF000E5040E944E058A810E94E5040E944E058D
:100B000022960FB6F894DEBF0FBECDBFDF91CF9116
:100B10000895CF93DF93CDB7DEB721970FB6F89442
:100B2000DEBF0FBECDBF8983A5E3B0E0E5E3F0E013
:100B3000808188608C9389810E94670521960FB619
:100B4000F894DEBF0FBECDBFDF91CF910895CF9354
:100B5000DF93CDB7DEB724970FB6F894DEBF0FBE94
:100B6000CDBF9C838B838B819C81DC01FD01019037
:100B70000020E9F73197CF018A1B9B0B8A831982EA
:100B80000EC0898199279C018B819C81F901E80F16
:100B9000F91F80810E94890589818F5F89839981EE
:100BA0008A81981770F324960FB6F894DEBF0FBEB3
:100BB000CDBFDF91CF910895CF93DF93CDB7DEB74F
:100BC00021970FB6F894DEBF0FBECDBF898381E0B9
:100BD00090E00E94AB04A5E3B0E0E5E3F0E08081A3
:100BE000877F8C9389810E946705A5E3B0E0E5E3E8
:100BF000F0E0808188608C9321960FB6F894DEBF78
:100C00000FBECDBFDF91CF910895CF93DF93CDB7C6
:100C1000DEB723970FB6F894DEBF0FBECDBF8A8331
:100C20006B838A81882319F48B81805889838A8118
:100C3000813019F48B818054898389810E94DC057D
:100C400023960FB6F894DEBF0FBECDBFDF91CF91D4
:100C50000895CF93DF93CDB7DEB781E090E00E9497
:100C6000AB04A5E3B0E0E5E3F0E08081877F8C93FF
:100C700083E00E94E5040E944E0585E090E00E941A
:100C8000AB0483E00E94E5040E944E0581E090E001
:100C90000E94AB0483E00E94E5040E944E0582E0BE
:100CA0000E94E5040E944E0581E090E00E94AB04A2
:100CB00088E20E94DC058EE00E94DC0581E00E9453
:100CC000DC0584E890E00E94A7056AE081E00E94CC
:100CD000050689E890E00E94A705DF91CF9108956D
:100CE000CF93DF93CDB7DEB722970FB6F894DEBF70
:100CF0000FBECDBF8091AC00882309F448C080911D
:100D0000AF00813009F041C08091AC00181634F476
:100D10008091B0008F5F8093B00005C08091B000DB
:100D200081508093B0008091B00088231CF482E051
:100D30008093B0008091B000833014F01092B00026
:100D40008091B000282F332727FD30953A832983DF
:100D500089819A818130910579F029813A81223007
:100D6000310579F089819A81009709F00EC060E021
:100D700080E00E94050609C069E080E00E94050647
:100D800004C060E081E00E9405061092AC0022964B
:100D90000FB6F894DEBF0FBECDBFDF91CF9108959F
:100DA000CF93DF93CDB7DEB781E08093AF00109291
:100DB000B0000E94A10460E080E00E9405068EE879
:100DC00090E00E94A70569E080E00E94050686E9A0
:100DD00090E00E94A70560E081E00E9405068DE991
:100DE00090E00E94A7050E948D0460E080E00E94D0
:100DF00005061092AC00DF91CF910895CF93DF9359
:100E0000CDB7DEB721970FB6F894DEBF0FBECDBFCA
:100E10001982F894E0E3F0E0808199278071907066
:100E2000009711F081E08983E0E3F0E08081992769
:100E300088709070009721F0898193E089278983D9
:100E40007894998180916900292F281B822F8983AA
:100E50008981992787FD909581709070882381F012
:100E600080916900982F8981890F80936900898119
:100E7000982F92708091AC00890F81508093AC00C4
:100E800021960FB6F894DEBF0FBECDBFDF91CF9194
:100E90000895FB019F01E8944230C4F04532B4F458
:100EA0004A3029F497FB1EF4909581959F4F642F4B
:100EB00077270E947A07805D8A330CF0895D8193E1
:100EC000CB010097A1F716F45DE251931082C9019E
:100ED0000C946A07DC01FC0101900020E9F73297CD
:100EE000AE17BF0730F47C916081708331976D93AA
:100EF000F7CF0895AA1BBB1B51E107C0AA1FBB1F58
:100F0000A617B70710F0A61BB70B881F991F5A9595
:0C0F1000A9F780959095BC01CD010895D3
:100F1C004B2000000000003D00010D0A4550492DFA
:100F2C005465737465720056657273696F6E203008
:100F3C002E3264006875687500416B6B75005050FB
:100F4C004D2D4F75740050504D2D496E00444D5829
:040F5C002D496E00AD
:00000001FF
